:100000000A308A00CF2A0000FF00030E8301A100FE
:100010000A08A0008A010408A2007708A300780853
:10002000A4007908A5007A08A600831383128C30F7
:100030008400801C1D288C1832288B1E21280B1947
:100040003528220884002308F7002408F800250832
:10005000F9002608FA0020088A00210E8300FF0E0E
:100060007F0E09008A110A12942D8A110A12EA2CB5
:100070000A108A100A11820728340C34013406341D
:10008000C822412A49274710C62049265529C510AC
:100090000000DE01DD01DF015F081F3C031C622858
:1000A0001F151F19512883161E088312DD071E080D
:1000B00003181E0FDE071030F700F70B5D28000055
:1000C000DF0A4C285E0CFA005D0CF900FA0CF90C02
:1000D000FA0CF90CFA0CF90CFA0CF90C0730FA05C9
:1000E0007908F8007A08F90008008E30F7005E08F9
:1000F000F8005D08F900FA01F808031D892879085D
:10010000F800F9010830F702F808031D8928F70103
:1001100091280310F81B9028F90DF80DF703892892
:10012000F81308006A0803190229F2006E0803197F
:100130000229F2070318A3287F30F202031C0229C8
:1001400003190229A7288130F2070318022972082F
:10015000F700F801F901FA016B08F600F6176C08D0
:10016000F5006D08F4001830F200F301741CD0287B
:100170007108FA07031CC228F90A031DC228F80AED
:100180000319F3177008F907031CC928F80A0319A3
:10019000F3176F08EC00EC176C08F8070318F31757
:1001A000F30DF80CF90CFA0CF60CF50CF40C03102A
:1001B000F20BB5280130F70703180229F81BE728CE
:1001C000F60DFA0DF90DF80DF70303190229F61FC4
:1001D000F828FA0A031DF828F90A031DF828F80A76
:1001E000031DF828F80CF90CFA0CF70A0319022978
:1001F0006B08F3006F08F306F31F0029F8170629B0
:10020000F8130629F701F801F901FA010800803016
:100210008318E806ED01EE016408EC006808EC06BE
:1002200063080319F729EB00F70067080319002A90
:10023000EB0203199C29031C5A296808F100F117E5
:100240006908F0006A08EF00EE010310F10CF00CF1
:10025000EF0CEE0CEB0B2429EC1F31296D14142A42
:100260006D106B106D16663084008313292A6D1291
:10027000EC1B44296B1C4F29F10CF00CEF0CEE0C1D
:10028000F70A03190F2A4F29F11B52290310EE0D0B
:10029000EF0DF00DF10DF70303190F2A44296D1727
:1002A000BC296D136408EC00EC1F5829F117082ACB
:1002B000F113082A6708EB00F7006308EB026408F3
:1002C000F100F1176508F0006608EF00EE01031079
:1002D000F10CF00CEF0CEE0CEB0B6629EC1F732904
:1002E000ED14142AED106B10ED166A3084008313A0
:1002F000292AED12EC1B86296B1C9129F10CF00CBC
:10030000EF0CEE0CF70A03190F2A9129F11B94291F
:100310000310EE0DEF0DF00DF10DF70303190F2A89
:100320008629ED17BC29ED136808EC00EC1F9A290B
:10033000F117082AF113082A6808F100F117690873
:10034000F0006A08EF00EC1FA929F1136D15142ABB
:100350006D11EE016B10663084008313292AEC1BAB
:10036000D2296408EC006B1CBC29F10CF00CEF0CDA
:10037000EE0CF70A03190F2AEE1FCD29EF0A031D11
:10038000CD29F00A031DCD29F10A031DCD29F10C59
:10039000F00CEF0CF70A03190F2A6D1B5129ED1B06
:1003A0009329F1298030F106F11FDA29142A68080F
:1003B000EC00E7296408EC00F108031DE729F008C8
:1003C000031DE729EF08031DE729F701082AF11BA0
:1003D000F1290310EE0DEF0DF00DF10DF70BE729EC
:1003E0000F2AEC1FF529F117082AF113082A6708CC
:1003F000F7006808F1006908F0006A08EF00082AB1
:100400006308F7006408F1006508F0006608EF0073
:100410007108F8007008F9006F08FA00472AF70120
:10042000F801F901FA01472AEE01EF09F009F10993
:10043000EE09EE0A031D222AEF0A031D222AF00A02
:100440000319F10A6D183029ED1872296D19A829C0
:10045000D7290008EF07031C332AF00A031D332AAB
:10046000F10A03196B1484030008F007031C3B2AEC
:10047000F10A03196B1484030008801F803AF10706
:1004800003186B146D1A3729ED1A7929AF29080062
:1004900049207908FA007808DD007908DE00752027
:1004A0007030ED009830EC002C30EB007E30EA002C
:1004B0007A08F1007908F0007808EF007708EE007C
:1004C00092207708DD007808DE007908DF007A08DE
:1004D000E000E2010408E1006210831B621483144F
:1004E0007A08E6007908E5007808E4007708E30078
:1004F000CD30EA002C30E9001330E8008730E70007
:1005000007216108840083136218831708006108BB
:1005100003194C2BED00650803194C2BED02031C4D
:10052000962A7F30ED0703184C2B9C2A8130ED0270
:10053000031C4C2B03194C2B6D08F700F801F90133
:10054000FA01EC016208EB00EB176308EA006408AB
:10055000E9001930ED006808E9020318BF2A0130EC
:10056000EA020318BF2AEB020318BF2AEC020318A1
:10057000BF2AEC0AEB0AEA0A6808E907F12A6708C9
:10058000EA020318DA2A0130EB020318DA2AEC0235
:100590000318DA2AEC0AEB0A6708EA076808E90791
:1005A000031CF12AEA0A031DF12AEB0A031DF12AB2
:1005B000EC0AF12A66088038EB020318F02A0130B1
:1005C000EC020318F02AEC0A66088038EB0767088B
:1005D000EA07031CCE2AEB0A031DCE2AEC0ACE2A18
:1005E0007A14ED0BF42AFF2A0310E90DEA0DEB0D46
:1005F000EC0D0310FA0DF90DF80DEE0DAB2A6E1C83
:10060000072B0310F80CF90CFA0CEE0C0A2BF7036D
:1006100003194C2BEE1B332B0310E90DEA0DEB0DE8
:10062000EC0D6808E90203181F2B0130EA020318D9
:100630001F2BEB0203181F2BEC02031C422B670835
:10064000EA0203182A2B0130EB0203182A2BEC02D2
:10065000031C422B66088038EB020318332B013051
:10066000EC02031C422BFA0A031D422BF90A031D5C
:10067000422BF80A031D422BF70A03194C2BF80CE6
:10068000F90CFA0C6208ED006608ED06ED1F4A2B26
:10069000F817502BF813502BF701F801F901FA0164
:1006A00008006008F8015F020318592B5F08F70083
:1006B000652BF7010830E100DF0DF70D60087702C8
:1006C0000318F700F80DE10B5C2B08008316861366
:1006D000831286130830F8006D2B0000F8177E2B6C
:1006E000F813EA0C03188617031C861378177E2B61
:1006F0007813F80B712B7C2B000086171C308400BC
:10070000840B802B832BF81B702B781B782B080015
:1007100078085D08DF006430E00051237708DD00D1
:1007200078083030031D9B2BDE1CA22BDE19A22B78
:100730005E1A20309E2BDE115E125E14F8077808D8
:10074000EA0066235D08DF000A30E00051237708E5
:10075000DD0078083030031DB32BDE19B72B5E1C8B
:10076000B72B5E1A2030F8077808EA00662330308D
:10077000DD075D08EA00662308006A08B63CEA0067
:10078000FA016B08EE00EB170310EB0CEC0CED0C10
:10079000FA0CF90CF80CF70CEA0BC42BEE1FDB2B50
:1007A000F709F809F909FA09F70A0319F80A031908
:1007B000F90A0319FA0A0800F701F801F901FA0128
:1007C000F201F301F401F501710870046F046E0485
:1007D00003191A2C2030F6000310EA0DEB0DEC0D76
:1007E000ED0DF20DF30DF40DF50D71087502031DFD
:1007F000032C70087402031D032C6F087302031D81
:10080000032C6E087202031C142C6E08F2026F088F
:10081000031C6F0FF3027008031C700FF4027108C1
:10082000031C710FF5020314F70DF80DF90DFA0D05
:10083000F60BEC2B72308400831308000408E200EE
:100840006108E40003193D2C6008ED005F08EC002E
:100850005E08EB005D08EA00F101F0012030EF00D6
:100860008230EE0092207A08E0007908DF007808F4
:10087000DE007708DD00E40B242C6008ED005F0843
:10088000EC005E08EB005D08EA00BD237A08E0009A
:100890007908DF007808DE007708DD00E01F5D2CB6
:1008A000E203E216DD09DE09DF09E009DD0A0319CA
:1008B000DE0A0319DF0A0319E00A3B30E9009A3027
:1008C000E800CA30E700E6010A30E40061080319D5
:1008D000E20A6008ED005F08EC005E08EB005D08CE
:1008E000EA006908F1006808F0006708EF00660890
:1008F000EE00DC230008DD00840A0008DE00840A24
:100900000008DF00840A0008E000FD308407F708D3
:10091000031D9D2C610A640203199D2C62080319B2
:100920009F2C0F3964020319972C0318CF2CE21B5C
:10093000CF2C621B9F2C2030CB2C2030E205E21EF6
:10094000AD2CE2126108031DE2037708E2002D30AE
:10095000EA0066236208F700E20161086402031DF1
:10096000BB2C7708E2002E30EA0066236208F7000D
:100970002030E20500303030E21ECB2CE21261085C
:10098000031DE2037708E2002D30EA0066236208C7
:10099000F700E2013030F7077708EA0066236908BC
:1009A000ED006808EC006708EB006608EA00F1015A
:1009B000F001EF010A30EE00DC237A08E900790843
:1009C000E8007808E7007708E600E40B692C8A1154
:1009D0000A12802D2C082E020318FB2CA8122808BE
:1009E000831687008312871228132808831687002E
:1009F00083120713072DA812280883168700831275
:100A000087162813280883168700831207170310F8
:100A10002D0D2E020318132D281228088316870087
:100A200083120712192D28122808831687008312B3
:100A300007162E08643C0319202DAE08031D892DCE
:100A400048227A08DC007908DB007808DA007708A9
:100A5000D90083145C08E6005B08E5005A08E4004E
:100A60005908E3003208EA003108E9003008E800DC
:100A70002F08E70007217708DD007808DE007908F5
:100A8000DF007A08E000E4007908E3007808E2007B
:100A90007708E1001730E800B730E7005130E60092
:100AA0007D30E50087227A08B6007908B50078081D
:100AB000B4007708B3005C08B2005B08B1005A08C4
:100AC000B0005908AF002A08DD000130DE0088239D
:100AD0002030EA0066232B08DD000130DE00882389
:100AE0002030EA006623893084005C08E0005B085F
:100AF000DF005A08DE005908DD000330E1001E2C3B
:100B00002030EA0066230D30EA0066230A30EA004E
:100B100066232E08C73C031C8F2DAE0A902DAE0114
:100B20000B118A110A122128DA012930D900B70ADB
:100B30003708183C0318CB2DB70102305907840041
:100B400083135A188317800A801BCB2D00083B3C67
:100B50000318CB2D02305907840083135A188317CA
:100B6000800101305907840083135A188317800AC3
:100B7000801BCB2D00083B3C0318CB2D01305907BF
:100B8000840083135A188317800159088400831343
:100B90005A188317800A8C108A110A1221285029AA
:100BA0004524C52054002328D222C822412A0D05FD
:100BB0000000A519AE18E60843102000A518AE18CD
:100BC000E608C31773102000D327C125201020107A
:100BD0000001A329CF20CB060A00A519AE18E6080C
:100BE00043102000D3274C2245290001A3294F267A
:100BF000C422D2060A00A519AE18E6084310200048
:100C0000A518AE18E608C31773102000A519AE1872
:100C1000E60843102000D2224626CF2BA021CF2663
:100C20005026452A4500C3274F26492747100D0562
:100C30000001A519AE18E60843102000A518AE184B
:100C4000E608C3177310200006340934093406344B
:100C500080348034803480340034A812280883160D
:100C600087008312871628132808831687008312AB
:100C7000071783168113091283129412A8122808E9
:100C8000831687008312281628088316870083128C
:100C9000A8112808831687000130831294000030C1
:100CA000831694000108C03905388100853083120D
:100CB00090004830F80006389200F9308316920010
:100CC00007309C00050885000330F700F70B662EFF
:100CD0001C0883120D1383169D01C03083128B04F0
:100CE00083168C1483128B1683161F149F101F15E6
:100CF0009F111F1383121F179F1383169F178312B1
:100D00001F140030F8001F08C73978049F008A15A7
:100D10000A12EE2A4D3084008313000803199E2E18
:100D20000130F800F701F70B932EF80B922E4A30A2
:100D3000F700F70B992E9C2E800B902E08000808C8
:100D4000F039D50053080F395504880007152811CC
:100D5000280883168700000083120711281128082D
:100D60008316870083120800D108031DB92E87104F
:100D7000BA2E8714A8102808831687008312D20E73
:100D80005208D3009F26D20E5208D3009F260D3062
:100D9000F700F70BC92E0800C830CD008A26F030C6
:100DA0008316880583128710A810280883168700E9
:100DB0008312071128112808831687008312B801AF
:100DC0003808023C031CEC2E0230CD008A2603308A
:100DD000D3009F26B80AE02E0D30F700F70BEE2E59
:100DE0000230D3009F260D30F700F70BF52EB80127
:100DF0003808023C031C082F38083820B900D101FC
:100E00003908D200B4260230CD008A26B80AF82E5E
:100E10008A150A12FD2A831603178C170C1400007A
:100E2000000083128C080319322F0D080313B80039
:100E300003170F080313B90003170C080313BA00B4
:100E40000130D1003A08D200B426380803178D00CB
:100E50000313390803178F008D0A03198F0A031330
:100E60000B2F031703138A150A12112B83168C10EC
:100E7000023083123B07840083133C1883178001E0
:100E80003B08840083133C188317800101303B0723
:100E9000840083133C188317800183168C148312FB
:100EA000080001304D02CF004E08023C031D5A2FAE
:100EB0004030CF074F088038D000D1015008D20011
:100EC000B42608004C080C3A03196D2F063A031992
:100ED000752F073A03197B2F802FD1010130D200E3
:100EE000B4260230CD008A268C2F0130CD0002308E
:100EF000CE0051278C2F0130CD00CE0051278C2FF2
:100F00004C081F3C031C862F0730CC050130D10054
:100F10004C08D200B4268C2F0800831603178C17B8
:100F20000C140000000083120C087F390319D12F24
:100F30000313BB0003170D080313BC0003170F08AE
:100F40000313BD003B08CC0062273C0803178D004B
:100F500003133D0803178F0083168C170C14000031
:100F6000000083120C0D0E0D7F390319D12F0313CE
:100F7000BB0003170D080313BC0003170F0803136E
:100F8000BD003B08CC0062273C0803178D0003130B
:100F90003D0803178F008D0A03198F0A03138D2F45
:100FA000031703130800F701F8013F080310401866
:100FB000F707F70CF80CC018F707F70CF80C4019F6
:100FC000F707F70CF80CC019F707F70CF80C401AE4
:100FD000F707F70CF80CC01AF707F70CF80C401BD2
:100FE000F707F70CF80CC01BF707F70CF80C080014
:10100000831603178C170C140000000083120C08C1
:101010007F39031954280313BB0003170D0803136A
:10102000BC0003170F080313BD00A7018B1BA717F4
:101030008B133B08EA008A1166238A15A71B8B17BE
:101040003C0803178D0003133D0803178F00831618
:101050008C170C140000000083120C0D0E0D7F394C
:10106000031954280313BB0003170D080313BC0016
:1010700003170F080313BD00A7018B1BA7178B13C2
:101080003B08EA008A1166238A15A71B8B173C08C8
:1010900003178D0003133D0803178F008D0A0319F2
:1010A0008F0A031300280317031308004508CC0018
:1010B0004908CC06CC1F612803110310C51B03147B
:1010C00094284508CC004808CD004408CD020319F7
:1010D0006F28CC1F94280308013A830094284908FC
:1010E000CD004508CD0203197B28CC1F94280308A6
:1010F000013A830094284A08CD004608CD0203191E
:101100008728CC1F94280308013A830094284B08B1
:10111000CD004708CD0203199328CC1F942803085B
:10112000013A83009428031008008314A7018B1B45
:10113000A7178B133608E6003508E5003408E400ED
:101140003308E3003E08EA003D08E9003C08E800F7
:101150003B08E7008A1107218A15A71B8B177A081D
:10116000C3007908C2007808C1007708C0004308AE
:10117000C7004208C6004108C5004008C400CB01B2
:10118000CA01C901C8015620031CCC283C303F07C6
:10119000AC006430AD00CE28AC01AD0108000408FD
:1011A000C4004308C6000319F628A7018B1BA71724
:1011B0008B134208ED004108EC004008EB003F08AB
:1011C000EA00F101F0012030EF008230EE008A11D8
:1011D00092208A15A71B8B177A08C2007908C100D4
:1011E0007808C0007708BF00C60BD528A7018B1B65
:1011F000A7178B134208ED004108EC004008EB00F4
:101200003F08EA008A11BD238A15A71B8B177A08AD
:10121000C2007908C1007808C0007708BF00C21F6B
:101220001E29C403C416BF09C009C109C209BF0AE7
:101230000319C00A0319C10A0319C20A3B30CB00C3
:101240009A30CA00CA30C900C8010A30C600430833
:101250000319C40AA7018B1BA7178B134208ED00C3
:101260004108EC004008EB003F08EA004B08F100A1
:101270004A08F0004908EF004808EE008A11DC2314
:101280008A15A71B8B170008BF00840A0008C0003E
:10129000840A0008C100840A0008C200FD308407E7
:1012A000F708031D6629430A460203196629440804
:1012B000031968290F394602031960290318A02968
:1012C000C41BA029441B682920309A292030C4055A
:1012D000C41E7829C4124308031DC4037708C40040
:1012E0002D30CC008A1162278A154408F700C4010A
:1012F00043084602031D88297708C4002E30CC001D
:101300008A1162278A154408F7002030C40500308E
:101310003030C41E9A29C4124308031DC403770841
:10132000C4002D30CC008A1162278A154408F700CA
:10133000C4013030F7077708CC008A1162278A157C
:10134000A7018B1BA7178B134B08ED004A08EC0075
:101350004908EB004808EA00F101F001EF010A300A
:10136000EE008A11DC238A15A71B8B177A08CB00A5
:101370007908CA007808C9007708C800C60B2A296E
:101380000800831603178C170C14000000000318C4
:10139000F22983120C087F390313C00003170D08CC
:1013A0000313C10003170F080313C2004008CC0049
:1013B0008A1162278A15410803178D00031342081A
:1013C00003178F0083168C170C1400000000831283
:1013D0000313BF0BEC29EF2983160317F229132AF5
:1013E0008316031783120C0D0E0D7F390313C000F3
:1013F00003170D080313C10003170F080313C200DE
:101400004008CC008A1162278A15410803178D0015
:101410000313420803178F008D0A03198F0A031064
:101420000313BF0BC12908007808A7018B1BA7175E
:101430008B133B08DF006430E0008A1151238A15CA
:10144000A71B8B177708BB0078083030031D2F2AA5
:10145000BC1C382ABC19382A3C1A2030322ABC114C
:101460003C123C14F8077808CC008A1162278A15D0
:10147000A7018B1BA7178B133B08DF000A30E00086
:101480008A1151238A15A71B8B177708BB00780890
:101490003030031D512ABC19572A3C1C572A3C1ACC
:1014A0002030F8077808CC008A1162278A1530307E
:1014B000BB073B08CC008A1162278A1508008E30D2
:1014C000F7004008F8003F08F900FA01C01F6D2A34
:1014D000F809F909F90A0319F80AF808031D7A2A24
:1014E0007908F800F9010830F702F808031D7A2A94
:1014F000F701832A0310F81B812AF90DF80DF70371
:101500007A2AC01FF81308008E30F7003B08F70254
:101510003C08F9003D08F800F917F70803199B2A61
:101520000310F908031D972AF80803199B2AF90CE0
:10153000F80CF70B902ABC1FA22AF809F909F80A3F
:101540000319F90A0800A7018B1BA7178B138A112F
:1015500048228A15A71B8B177708BF007808C000A0
:101560007908C1007A08C2003E08C7003D08C600DD
:101570003C08C5003B08C4004208CB004108CA0033
:101580004008C9003F08C8005620031CCA2AAC0105
:10159000AD01CE2A4630AC005030AD0008008401C9
:1015A00083131F3083058316861383128617AC01BD
:1015B000AD01B201B101B001AF01B601B501B40195
:1015C000B301B70183161F149F141F159F11073015
:1015D0009C00FF308312A8008A112D2E8A15A812B4
:1015E0002808831687008312871628132808831675
:1015F0008700831207178A11CC2E8A15D101483033
:10160000D2008A11B4268A150230CD008A118A26AA
:101610008A15243003178D0006308F008A110313BA
:101620000B2F8A15D1010330D2008A11B4268A15F6
:101630000230CD008A118A268A15BC012930BB00F0
:101640008A1136278A150230B8009630CD008A11EB
:101650008A268A15B80B252BBC012930BB008A11BC
:1016600036278A150130CD000230CE008A1151276D
:101670008A15CF3003178D0005308F008A110313B0
:101680008D278A15D33003178D0005308F00031383
:101690000020BE01BD014030BC008030BB00BF0156
:1016A00095200130CD00CE008A1151278A15A7015F
:1016B0008B1BA7178B138A1148228A15A71B8B1720
:1016C0007708BB007808BC007908BD007A08BE0026
:1016D000023084007A08C2007908C1007808C0008E
:1016E0007708BF000130C300CF20DB3003178D0027
:1016F00005308F00031404300313BF00C1210C30E8
:10170000CD000130CE008A1151278A152A08BB006E
:101710000130BC0014223A30CC008A1162278A15AD
:101720002B08BB000130BC0014220A30CD0002306F
:10173000CE008A1151278A15893084003608C200EC
:101740003508C1003408C0003308BF000130C300B1
:10175000CF20E03003178D0005308F0003140630D2
:101760000313BF00C121C830CD008A118A268A1513
:10177000AA1BD12B2A08043C0318D12BAC01AD01C4
:101780000130CD000230CE008A1151278A15403039
:1017900003178D0000308F008A1103138D278A15DF
:1017A000D02BA7018B1BA7178B138A1148228A15F0
:1017B000A71B8B177708BB007808BC007908BD0011
:1017C0007A08BE00C7003D08C6003C08C5003B08BB
:1017D000C400CB01CA012030C9008630C8005620A1
:1017E0000318492BBC012930BB008A1136278A1502
:1017F0000130B9003908BF003C30C0008A11D3273E
:101800008A157808C001BF00BF1BC0035F22831484
:10181000A7018B1BA7178B13E601E5014830E400F5
:101820008530E3007A08EA007908E9007808E800E2
:101830007708E7008A1107218A15A71B8B177A08FA
:10184000BE007908BD007808BC007708BB00842280
:101850007808BA000C30CC008A1162278A15013052
:10186000CD000230CE008A1151278A15E4300317CB
:101870008D0005308F008A1103138D278A15E930FA
:1018800003178D0005308F0003130020BA08031DD5
:101890004C2CB9080319A12DBE01BD012030BC009C
:1018A0008630BB00A3220130CD00CE008A11512723
:1018B0008A15A7018B1BA7178B138A1148228A153B
:1018C000A71B8B177708BB007808BC007908BD0000
:1018D0007A08BE00023084007A08C2007908C1008C
:1018E0007808C0007708BF000130C300CF20EF3078
:1018F00003178D0005308F00031404300313BF005D
:10190000C1212B08BA02BA1F872C3B30BA002A0823
:10191000BF003C30C0008A11D3278A157808C00167
:10192000BF00BF1BC0035F228314A7018B1BA71737
:101930008B13E601E5014830E4008530E3007A08C6
:10194000EA007908E9007808E8007708E7008A11DA
:1019500007218A15A71B8B177708BB007808BC00E6
:101960007908BD007A08BE00C0012B08BF00BF1B6C
:10197000C0035F228314A7018B1BA7178B133E089C
:10198000E6003D08E5003C08E4003B08E3007A0877
:10199000EA007908E9007808E8007708E7008A118A
:1019A00007218A15A71B8B177708BB007808BC0096
:1019B0007908BD007A08BE00A7018B1BA7178B13FF
:1019C0007A08E4007908E3007808E2007708E1008B
:1019D000E801E7017030E6008430E5008A118722D3
:1019E0008A15A71B8B177A08BE007908BD007808F6
:1019F000BC007708BB0084227808B9002A08BF0021
:101A00003C30C0008A11D3278A157808C001BF0076
:101A1000BF1BC0035F228314A7018B1BA7178B1367
:101A2000E601E5014830E4008530E3007A08EA0089
:101A30007908E9007808E8007708E7008A110721AB
:101A40008A15A71B8B177708BB007808BC0079089C
:101A5000BD007A08BE00C0012B08BF00BF1BC00339
:101A60005F228314A7018B1BA7178B133E08E60088
:101A70003D08E5003C08E4003B08E3007A08EA0082
:101A80007908E9007808E8007708E7008A1107215B
:101A90008A15A71B8B177708BB007808BC0079084C
:101AA000BD007A08BE003908BF003C30C0008A1172
:101AB000D3278A157808C001BF00BF1BC0035F226F
:101AC0008314A7018B1BA7178B133E08E6003D0864
:101AD000E5003C08E4003B08E3007A08EA007908E6
:101AE000E9007808E8007708E7008A1107218A15DD
:101AF000A71B8B177A08BE007908BD007808BC00C8
:101B00007708BB0084227808BA000930CD00013084
:101B1000CE008A1151278A153908BB000130BC005C
:101B200014223A30CC008A1162278A153A08BB0089
:101B30000130BC001422C830CD008A118A268A15D3
:101B4000462CBC012930BB008A1136278A150C307F
:101B5000CC008A1162278A150130CD000230CE00F8
:101B60008A1151278A15F23003178D0005308F0036
:101B70008A1103138D278A15F63003178D0005305F
:101B80008F0003130020BE01BD012030BC00803057
:101B9000BB000A30BF0095200130CD00CE008A1175
:101BA00051278A15A7018B1BA7178B138A1148226F
:101BB0008A15A71B8B177708BB007808BC0079082B
:101BC000BD007A08BE00023084007A08C20079089D
:101BD000C1007808C0007708BF000130C300CF20E3
:101BE000FD3003178D0005308F00031404300313FC
:101BF000BF00C1210C30CD000130CE008A11512729
:101C00008A152A08BB000130BC0014223A30CC00EF
:101C10008A1162278A152B08BB000130BC001422F0
:101C20000A30CD000230CE008A1151278A15893042
:101C300084003608C2003508C1003408C0003308EB
:101C4000BF000130C300CF20023003178D000630E3
:101C50008F00031406300313BF00C121C830CD002C
:101C60008A118A268A15AA1B4C2E2A08023C0318C0
:101C70004C2EAC01AD010130CD000230CE008A11F6
:101C800051278A15403003178D0000308F008A11CC
:101C900003138D278A154B2EA7018B1BA7178B13B8
:101CA0008A1148228A15A71B8B177708BB00780872
:101CB000BC007908BD007A08BE00C7003D08C60018
:101CC0003C08C5003B08C400CB01CA015830C9001C
:101CD0008630C80056200318C32DBA08031D732E82
:101CE000B9080319182FBE01BD015830BC00863059
:101CF000BB00A3220130CD00CE008A1151278A15E6
:101D0000A7018B1BA7178B138A1148228A15A71BC3
:101D10008B177708BB007808BC007908BD007A08EB
:101D2000BE00023084007A08C2007908C100780839
:101D3000C0007708BF000130C300CF200830031770
:101D40008D0006308F00031404300313BF00C1213F
:101D50002B08BA02BA1FAE2E3B30BA002A08BF00C9
:101D60003C30C0008A11D3278A157808503CF8000F
:101D70002B087802BC003C08BD003C30BE003D088A
:101D80003E068039C000BD1FC72EBD09BD0ABE1F5B
:101D9000CB2EBE09BE0A3E08F8013D020318D32E21
:101DA0003D08F700DF2EF7010830BF00BD0DF70D2D
:101DB0003E0877020318F700F80DBF0BD62EC01FA0
:101DC000E32EF809F80A7808B9002A08BF003C3069
:101DD000C0008A11D3278A157808503CF8002B08D8
:101DE0007802BB003908BF003C30C0008A11D327FD
:101DF0008A1578083B02BA000930CD000130CE00C8
:101E00008A1151278A153908BB000130BC00142201
:101E10003A30CC008A1162278A153A08BB0001309B
:101E2000BC001422C830CD008A118A268A156D2E76
:101E3000AC01AD010C30CC008A1162278A1501304B
:101E4000CD000230CE008A1151278A150B300317BE
:101E50008D0006308F008A1103138D278A151330E9
:101E600003178D0006308F00031300200130CD00D2
:101E7000CE008A1151278A15A7018B1BA7178B1338
:101E80008A1148228A15A71B8B177708BB00780890
:101E9000BC007908BD007A08BE00023084007A08D0
:101EA000C2007908C1007808C0007708BF0001307F
:101EB000C300CF201B3003178D0006308F000314A2
:101EC00004300313BF00C1210A30CD000130CE0021
:101ED0008A1151278A15893084003608C2003508D6
:101EE000C1003408C0003308BF000130C300CF2058
:101EF000203003178D0006308F00031406300313C3
:0A1F0000BF00C121362F232B630020
:02400E003A3F37
:00000001FF
